:020000040800F2
:10000000400D002065010008630F0008490B00083F
:1000100000000000000000000000000000000000E0
:10002000000000000000000000000000851600082D
:100030000000000000000000591200088D180008A0
:1000400077010008770100087701000877010008B0
:1000500077010008A106000877010008C50600081E
:100060007701000877010008770100081D050008E6
:100070007701000877010008770100087701000880
:1000800077010008770100080000000077010008F0
:100090007701000877010008770100087701000860
:1000A000770100087701000877010008311900087E
:1000B0007701000800000000770100080000000040
:1000C00000F002F800F03EF80CA030C80838241800
:1000D0002D18A246671EAB4654465D46AC4201D180
:1000E00000F030F87E460F3E0FCCB6460126334274
:1000F00000D0FB1AA246AB4633431847D424000075
:10010000F4240000103A02D378C878C1FAD8520714
:1001100001D330C830C101D504680C6070470000BD
:100120000023002400250026103A01D378C1FBD813
:10013000520700D330C100D50B6070471FB51FBDFB
:1001400010B510BD00F01CF91146FFF7F7FF01F0E4
:1001500051FE00F034F903B4FFF7F2FF03BC00F0E6
:100160003BF900000748804707480047FEE7FEE7E5
:10017000FEE7FEE7FEE7FEE704480549054A064BB1
:1001800070470000B5180008C100000840070020B3
:10019000400D0020400900204009002030B5441CDB
:1001A00003E00178401C00290DD08107F9D10B4BE9
:1001B000DD0104C8D11A91432940FAD0001B0A0678
:1001C00003D0C01E30BD001B30BD0A0401D0801E0C
:1001D00030BD0902FCD0401E30BD0000010101010C
:1001E00001E004C0091F0429FBD28B0701D502805E
:1001F000801CC90700D00270704700290BD0C307CC
:1002000002D00270401C491E022904D3830702D584
:100210000280801C891EE3E70022EEE70022DFE770
:10022000002203098B422CD3030A8B4211D30023F3
:100230009C464EE003460B433CD4002243088B42CD
:1002400031D303098B421CD3030A8B4201D394465A
:100250003FE0C3098B4201D3CB01C01A524183094D
:100260008B4201D38B01C01A524143098B4201D307
:100270004B01C01A524103098B4201D30B01C01A32
:100280005241C3088B4201D3CB00C01A52418308AC
:100290008B4201D38B00C01A524143088B4201D3D9
:1002A0004B00C01A5241411A00D201465241104639
:1002B00070475DE0CA0F00D04942031000D34042AE
:1002C000534000229C4603098B422DD3030A8B42E4
:1002D00012D3FC22890112BA030A8B420CD3890182
:1002E00092118B4208D3890192118B4204D3890168
:1002F0003AD0921100E08909C3098B4201D3CB01A6
:10030000C01A524183098B4201D38B01C01A52415A
:1003100043098B4201D34B01C01A524103098B425E
:1003200001D30B01C01A5241C3088B4201D3CB0049
:10033000C01A524183088B4201D38B00C01A52412C
:10034000D9D243088B4201D34B00C01A5241411A03
:1003500000D20146634652415B10104601D3404231
:10036000002B00D54942704763465B1000D34042E2
:1003700001B50020C046C04602BD704770477047B7
:10038000754600F025F8AE46050069465346C0089C
:10039000C000854618B020B5FFF7EEFE60BC002710
:1003A0004908B6460026C0C5C0C5C0C5C0C5C0C541
:1003B000C0C5C0C5C0C5403D49008D46704710B599
:1003C0000446C046C0462046FFF7C5FE10BD0000EB
:1003D00000487047DC06002001491820ABBEFEE74C
:1003E000260002007047000038B50021009100246B
:1003F0006A460F4801F0B4FB68460078002815D122
:1004000001F03CFD002811D000BF0CE0204601F0B7
:1004100041FD002805D0E100064A89184868804758
:1004200003E0601CC4B20D2CF0DB00BF38BD00003F
:1004300048060020F4240008054800880549884241
:1004400004D003480088401C014908807047000020
:1004500042000020FFFF000010B5002000F040FE29
:1004600004462078042805DA608822789200064B3A
:1004700099588847054800887D210901884202DB98
:1004800000200249088010BD5C25000842000020C1
:1004900010B54C220021024800F058FD10BD0000AC
:1004A0009006002010B51A48C079012822D11948B9
:1004B0000078401C1749087008460078052804DABF
:1004C0001021154800F020FA21E012480078092890
:1004D00007DB00200F49087010210F4800F012FAC6
:1004E00015E00C480078052811DD10210A4800F0BD
:1004F00009FA0CE00648C079022804D11021064808
:1005000000F002FA03E01021034800F0FBF910BDEF
:10051000D00600203C0000200004004810B5012057
:10052000800300F0D7F8002803D00120800300F0FA
:10053000CBF810BD10B55748807D002804D180212C
:10054000554800F0DFF92EE05248807D012804D1A3
:100550008021514800F0D8F925E04E48807D0228DE
:1005600021D14E480078401C4C490870084600785C
:10057000052804DA8021484800F0C6F913E047480E
:100580000078092807DB0020444908708021424890
:1005900000F0B8F907E041480078052803DD802124
:1005A0003D4800F0AFF93B4816304078002804D1B0
:1005B0004021394800F0A6F930E03648163040783E
:1005C000012804D14021344800F09EF926E031484A
:1005D00016304078022821D130484078401C2F49FD
:1005E000487008464078052804DA40212A4800F07F
:1005F0008BF913E029484078092807DB00202749B8
:1006000048704021244800F07DF907E023484078F5
:10061000052803DD4021204800F074F91D481630FC
:100620008078002804D120211B4800F06BF930E0CD
:10063000184816308078012804D12021164800F08F
:1006400063F926E0134816308078022821D1134838
:100650008078401C1149887008468078052804DAA3
:1006600020210D4800F050F913E00C48807809284B
:1006700007DB0020094988702021074800F042F973
:1006800007E006488078052803DD2021024800F0B5
:1006900039F910BDB00600200004004838000020E1
:1006A00010B5012000F016F8002802D0012000F05B
:1006B0000BF8022000F00EF8002802D0022000F013
:1006C00003F810BD70470000014948617047000001
:1006D0000004014001460020044A52690A40002AF1
:1006E00001D0012000E0002070470000000401401C
:1006F000002120498279002A35D00A461268036811
:100700009A430B461A600A46526803689A430B469E
:100710005A60027951180A6803681A430A60154A38
:10072000926803689A43134B9A601A46D26803682A
:100730009A43104BDA604279102A0CD11A4692681B
:1007400003681A430B4B9A601A46D26803681A432F
:10075000084BDA600DE00749427951180A680368CE
:100760001A430A6005E0027951180A6803689A433F
:100770000A6070470004014000B585B001214804BB
:1007800000F02CFE0121880500F028FE012108461A
:1007900000F044FE012080020090012168460171B2
:1007A000002181710121C17169460920C00600F054
:1007B00035F8012189020920C00600F0A5F80120C2
:1007C000009000216846017101218171032141716E
:1007D0000121C17169460F4800F020F80021052071
:1007E00000F052FF012003900021684601740C21A3
:1007F00041740121817403A8FFF77AFF052168463F
:100800000172002141720121817202A800F0AAFB4D
:1008100005B000BD0014004870477047F0B50A46A7
:1008200000210023002400BF3DE001258D402B4620
:1008300015681D402C469C4234D11579012D02D0FB
:100840001579022D16D185684F000326BE40B543A9
:10085000856055794E00B54086683543856085884A
:1008600001268E40B5438580858896798E40B6B244
:100870003543858005684F000326BE40B5430560BB
:1008800015794E00B540066835430560C5684F00D0
:100890000326BE40B543C560D5794E00B540C66855
:1008A0003543C560491C1029BFD3F0BDF0B5002306
:1008B00000244D07EE0E1546B5402B46CD10AE0078
:1008C00005462035AD594E07F70E0F26BE40B543FD
:1008D000CE10B60007462037BD51CD10AE003D46C4
:1008E000AD591D432C46CD10AD003E467451F0BDB0
:1008F00002460020138A0B40002B01D0012000E0AB
:100900000020704701857047816170471CB5012147
:100910000720400400F062FD0121880500F05EFD23
:100920000121084600F07AFD01200090012168466F
:10093000017103214171002181710121C171694659
:100940000920C006FFF76AFF402000900121684699
:10095000017103214171002181710121C171694639
:100960000920C006FFF75AFF40210920C006FFF703
:10097000C9FF80200090002168460171012181712A
:10098000032141710121C17169460920C006FFF7A9
:1009900045FF01200090002168460171012181710D
:1009A000032141710121C17169466648FFF736FF95
:1009B000022000900021684601710121817103210C
:1009C00041710121C17169465E48FFF727FF01208F
:1009D00040020090002168460171012181710321CC
:1009E00041710121C17169460920C006FFF716FF58
:1009F000012080020090002168460171012181716F
:100A0000032141710121C17169460920C006FFF728
:100A100005FF0120C00200900021684601710121FC
:100A20008171032141710121C17169460920C0060C
:100A3000FFF7F4FE012000030090002168460171D9
:100A400001218171032141710121C1716946092090
:100A5000C006FFF7E3FE0120C003009001216846B5
:100A6000017103214171002181710121C171694628
:100A70000920C006FFF7D2FE0121C9030920C006E4
:100A8000FFF740FF08200090012168460171032113
:100A90004171002181710121C17169462948FFF727
:100AA000BDFE08212748FFF72DFF102000900121EF
:100AB0006846017103214171002181710121C171D9
:100AC00069462048FFF7AAFE10211E48FFF71AFFCB
:100AD000202000900121684601710321417100210D
:100AE00081710121C17169461648FFF797FE2021E7
:100AF0001448FFF707FF402000900121684601716C
:100B000003214171002181710121C17169460D48A4
:100B1000FFF784FE40210B48FFF7F4FE8020009091
:100B20000121684601710321417100218171012178
:100B3000C17169460348FFF771FE80210148FFF744
:100B4000E1FE1CBD0004004800BFFEE70148024969
:100B500008607047CCCC00000030004001480249DA
:100B600008607047AAAA00000030004001494860B0
:100B70007047000000300040014988607047000065
:100B8000003000400149086070470000003000401C
:100B90001CB5002400200090019001218902092049
:100BA000C006FFF7A5FE002801D1012000E00020CB
:100BB0006946087001216148FFF79AFE002801D1BB
:100BC000012000E000206946487080210920C0060D
:100BD000FFF78EFE002801D1012000E000206946C9
:100BE0008870012109030920C006FFF781FE002853
:100BF00001D1012000E000206946C8700121C9022E
:100C00000920C006FFF774FE002801D1012000E092
:100C100000206946087102214848FFF769FE002854
:100C200001D1012000E000206946487101214902FC
:100C30000920C006FFF75CFE002801D1012000E07A
:100C4000002069468871002475E06846005D002830
:100C500039D13B48C07F0121A14088433849C8773A
:100C60000020384908553848005D401C3649085571
:100C700000206100354A50523348005D032858DD9A
:100C80000020314908553248005D6946095D8842B7
:100C90004FD02F48005D022808D1601D0002801C43
:100CA00082B20121002000F067FA07E0601D000217
:100CB000401C82B20121002000F05EFA6846005D0F
:100CC0002349085535E01E48C07F0121A140084353
:100CD000C1B21B48C1771B48005D401C194908552B
:100CE0000020194908551748005D032821DD002020
:100CF0001449085560001549085A1649884207DD0D
:100D00001348005D022814D002201149085510E054
:100D10000F48005D6946095D88420AD0601D0006E3
:100D2000020C0121002000F027FA6846005D084906
:100D30000855601CC4B2072C87DB1CBD00040048AA
:100D4000B00600201B0000202200002068000020C8
:100D500014000020DC0500007047000070B5054657
:100D600000242C120E4844720E2C04D110210D4880
:100D7000FFF7C8FD13E00D2C04D140210948FFF70F
:100D8000C3FD0CE00C2C04D180210648FFF7BCFD0C
:100D900005E00B2C03D120210248FFF7B5FD70BD03
:100DA000D00600200004004810B562480078401CBE
:100DB000604908706048407A6049097888427DD06F
:100DC00000205C4908705C48407A0D282DD15C48B1
:100DD0000078401C5A490870084600780A280CDD43
:100DE00058480078401C5749087000205449087042
:100DF00020215548FFF786FD0CE051480078052872
:100E000004DD20215048FFF77DFD03E020214E48FE
:100E1000FFF77AFD4B48007802286FDD0020494932
:100E2000087000214448417268E04348407A0C2829
:100E30002DD143480078401C41490870084600788D
:100E40000A280CDD3F480078401C3E49087000200D
:100E50003B49087020213C48FFF754FD0CE038481E
:100E60000078052804DD20213748FFF74BFD03E01B
:100E700020213548FFF748FD3248007800283DDD45
:100E800000203049087000212B48417236E02A4882
:100E9000407A0B282FD12A480078401C2849087036
:100EA000084600780A280EDD26480078401C2549AF
:100EB0000870002022490870202100E022E022482A
:100EC000FFF720FD0CE01E480078052804DD2021F6
:100ED0001D48FFF717FD03E020211B48FFF714FD15
:100EE00018480078002809DD002016490870002104
:100EF0001148417202E00020124908700E48407A01
:100F00000E4908700B480078322808DD0020094996
:100F10000870002108484172407A08490870064963
:100F20002039887C00F03CFCFFF704FBFFF7BAFA9D
:100F300010BD00003E000020D00600203D00002033
:100F40003F000020400000200004004830B5044667
:100F5000002303E02170641C5D1CABB29342F9DBFB
:100F600030BD704700218278002A27D0184A032319
:100F70001B02D21803789B109B00D158027892076D
:100F8000D30EFF229A400B469343194642789207AC
:100F9000120E03789B07DB0E9A4011430C4A032381
:100FA0001B02D21803789B109B00D1500278D30605
:100FB000DB0E01229A40064B1A6007E00278D30646
:100FC000DB0E01229A40024B80331A60704700000A
:100FD00000E100E010B5002819DA1A4A03071B0FD8
:100FE000083B9B089B00D2588307DC0EFF23A340DD
:100FF0009A438B071B0E8407E40EA3401A43114B40
:101000000407240F083CA408A4001A5118E00E4A53
:1010100003231B02D21883089B00D2588307DC0EDF
:10102000FF23A3409A438B071B0E8407E40EA340C3
:101030001A43054B032424021B198408A4001A51E7
:1010400010BD00001CED00E000E100E010B500283C
:1010500019DA1A4A03071B0F083B9B089B00D2585A
:101060008307DC0EFF23A3409A438B071B0E8407E4
:10107000E40EA3401A43114B0407240F083CA408B4
:10108000A4001A5118E00E4A03231B02D218830849
:101090009B00D2588307DC0EFF23A3409A438B07A3
:1010A0001B0E8407E40EA3401A43054B03242402BD
:1010B0001B198408A4001A5110BD00001CED00E0AB
:1010C00000E100E0002252214143044B5A548022A7
:1010D00052214143C9184A70704700007600002031
:1010E00070B5014600201C4D2870522048431B4D0E
:1010F000285C43065B0E5220484340194078420664
:10110000520E52204843401940788025284004461A
:10111000002C13D152204843104D4019801C9500DB
:1011200040190D4D06882E8040886880501CC2B240
:10113000142A00DB0022934200D10124002C01D0AC
:101140008020024352204843044D2B5452204843F0
:1011500040194270004870BD2A000020760000202F
:1011600010B5002404E02046FFF7ACFF601CC4B2B9
:10117000072CF8DB10BD0000F8B50B466E46337047
:101180007280522646431A4FBE5D7106490E5226A2
:101190004643BE5D80273E40354652264643144FA7
:1011A000F61976787406640E002D13D15226464344
:1011B000F619B61C8F00F7196E4636883E806E46CB
:1011C00076887E804E1CF1B2142900DB0021A142FA
:1011D00000D10125002D01D08026314352264643FF
:1011E000034FB95552264643F6197470F8BD0000F6
:1011F0007600002010B502460020154B18688008C4
:101200008000034613431846114B1860114B1B69AD
:10121000042423430F4C2361012907D130BF234607
:101220001B690424A3430B4C23610FE0022907D15F
:1012300020BF084B1B690424A343064C236105E02F
:10124000044B1B6902242343024C236110BD0000A0
:101250000070004000ED00E07047000010B5474806
:101260000078030000F0B8FD09060E1D2A323B4746
:101270004855870041480078401C404908700020CC
:10128000488079E03D4840887D21C900884200DCE3
:1012900072E000203949488008460078401C0870F8
:1012A0006AE0364840887D210901884200DC63E01D
:1012B00032480078401C314908705DE000202F4919
:1012C000488008460078401C087055E000202B49F3
:1012D000C880488008460078401C08704CE02748C9
:1012E00040882749884200DC46E024480078401CBA
:1012F0002249087040E03FE0204840887D21C90035
:10130000884200DC38E000201C4948800820087032
:1013100032E01A484088642800DA2DE0FFF72CFA02
:1013200000F0B8FA00F0C6FA0120164948707D2195
:10133000C90015480068FEF773FF0446601E134994
:10134000884201D901200CE0601E11494861032147
:10135000081FFFF73FFE00200D4988610720086144
:101360000020002801D000BFFEE7052003490870D7
:101370000020488000E000BF00BF10BDB402002084
:10138000881300009006002000000020FFFFFF00EF
:1013900000E000E00A4840880A49884204D0084832
:1013A0004088401C064948800548C0880549884255
:1013B00004D00348C088401C0149C8807047000021
:1013C000B4020020FFFF000000200349087048809D
:1013D00008718860C8807047B4020020002905D0D9
:1013E000054A52690243044B5A6104E0024A5269B9
:1013F0008243014B5A61704700100240002905D01A
:10140000054AD2690243044BDA6104E0024AD26918
:101410008243014BDA61704700100240002905D079
:10142000054A92690243044B9A6104E0024A9269B8
:101430008243014B9A61704700100240FEB504469A
:101440000025002600200290019000900027864889
:1014500040680C2108400546002D06D0042D07D019
:10146000082D08D00C2D2CD128E0804820602BE0DE
:101470007E48206028E07C4840680F2189040840AD
:101480000646794840680321C90308400290B00C21
:10149000861C0298002803D17548374647430BE065
:1014A0007148C06A0007000F401C01906F48019905
:1014B000FEF7B6FE70430746276005E06D482060E2
:1014C00002E06A48206000BF00BF67484068F02122
:1014D000084005462D096848405D00902068009945
:1014E000C84060606048406807210902084005461E
:1014F0002D0A6148405D009061680098C140A1607C
:101500005948006BFF2101310840884202D05B48F6
:10151000E0600DE05448406801218903084088429A
:1015200003D0A0684008E06002E0A0688008E060A6
:101530004D48006B40210840402802D050482061AF
:1015400002E00120C00320614748006B10210840E1
:10155000102802D04548606101E02068606142487F
:10156000006B8007800F002802D1A068A06119E0FD
:101570003D48006B8007800F012802D12068A061E0
:1015800010E03948006B8007800F022802D18003E9
:10159000A06107E03448006B8007800F032801D169
:1015A0003248A0613048006B03210904084000283C
:1015B00002D1A068E06120E02B48006B0321090400
:1015C000084001210904884202D12068E06114E04A
:1015D0002548006B03210904084001214904884281
:1015E00002D18010E06108E01F48006B032109046C
:1015F0000840884201D11D48E0611B48006B03216F
:1016000089040840002802D1A068206220E0164822
:10161000006B03218904084001218904884202D11A
:101620002068206214E01048006B03218904084000
:101630000121C904884202D10011206208E00A4851
:10164000006B032189040840884201D107482062C9
:101650000548006B80210840802802D00548606260
:1016600000E06762FEBD00000010024000127A0038
:1016700000093D00006CDC0258000020809FD5006E
:10168000128000007047000030B500228B071C0F4D
:101690000F23A3401A460B4B8C10A4001B599343F5
:1016A000084C8D10AD00635123468C10A4001B59CB
:1016B0008C07250F0446AC402343024C8D10AD002F
:1016C000635130BD080001400CB50020019000902E
:1016D000304800680121090408432E49086000BF12
:1016E0002C48006801214904084000900198401CE2
:1016F00001900098002803D1274901988842EFD132
:1017000024480068012149040840002802D0012033
:10171000009001E0002000900098012839D11120AC
:101720001E4908601B4840681A49486008464068DE
:101730004860084640687F21C903884315494860CE
:1017400008464068112109040843124948600846C8
:1017500000680121090608430E49086000BF0D48D2
:1017600000680121490608400028F8D0094840686F
:101770008008800007494860084640680221084305
:101780000449486000BF034840680C21084008280D
:10179000F9D10CBD00100240FFFF00000020024004
:1017A00010B50446002C05D140210920C006FFF7E2
:1017B000ABF82EE0012C05D140210920C006FFF72F
:1017C000A1F826E0022C24D112480078401C1149CF
:1017D000087008460078052805DA40210920C0066F
:1017E000FFF790F815E00B480078092808DB402146
:1017F0000920C006FFF788F800200649087008E0B5
:1018000004480078052804DD40210920C006FFF7C0
:101810007BF810BD3700002010B517480078FF286E
:1018200004D015480078401C13490870134800780C
:10183000FF2804D011480078401C10490870104857
:101840000078FF2804D00E480078401C0C4908702E
:101850000C480078FF2804D00A480078401C094949
:101860000870FFF797FDFEF7E7FD07480078401C7A
:101870000549087010BD0000320000203300002030
:1018800034000020350000203600002010B5FFF79E
:10189000C3FF10BD10B50020054908618861012112
:1018A0000807FFF7ABFD01210846FFF7A3FC10BDB9
:1018B00000E000E010B51B48006801210843194909
:1018C00008600846406818490840164948600846BC
:1018D000006816490840134908600846006801215D
:1018E000890488430F490860084640683F2109047D
:1018F00088430C4948600846C06A00090001C86274
:101900000846006BFF2154318843064908630846A6
:10191000406B40084000486300208860FFF7D4FE19
:1019200010BD0000001002400CB8FFF8FFFFF6FEEB
:1019300010B500F047F910BD01627047002904D0CE
:10194000026801231A43026003E002685208520051
:101950000260704702460020D3690B40002B01D083
:10196000012000E000207047F8B50346002400265F
:1019700000960025002018460E04340ECEB20096C4
:101980000127009EB7403D46022C01D1001D02E018
:10199000032C00D10830002A03D006682E430660CD
:1019A00002E00668AE430660F8BD0000F0B58BB0FB
:1019B00004460D46002700200A90002620684008B3
:1019C00040002060666803210903304688430646CC
:1019D000A8680643666026682D480640E96868687E
:1019E00008432969084306432660A66803210902C3
:1019F00030468843064668690643A6606846FFF796
:101A00001DFD2448844202D106980A900DE0224828
:101A1000844202D107980A9007E02048844202D10C
:101A200008980A9001E002980A9020680121C903F1
:101A3000084000280CD029680A9A5000FEF7F0FBF5
:101A4000074629680A9A5000FEF7EAFB0E4609E0AD
:101A500029680A98FEF7E4FB074629680A98FEF70A
:101A6000DFFB0E4628684008B04200D87F1C206883
:101A70000121C9030840002806D03807460F384620
:101A80000749084030430746A7810BB0F0BD00006E
:101A9000F3E9FFFF003801400044004000480040E7
:101AA000F0FF00000146888CC005C00D7047CA05D4
:101AB000D20D02857047000000B589B0182101A839
:101AC000FEF7ACFB00F080FA01214804FFF786FC2A
:101AD00001218803FFF7A2FC012202210920C00690
:101AE000FEF7E4FE012203210920C006FEF7DEFE18
:101AF0000C200790022108A80170032141700121E8
:101B00008170C17007A90920C006FEF787FEE12099
:101B100040020190002002900390049006900C2057
:101B2000059001A90B48FFF741FF01210948FFF784
:101B300005FF012208490748FFF716FF0122074960
:101B40000448FFF711FF40210248FFF7F5FE09B0F6
:101B500000BD000000380140050105000601060037
:101B6000F7B50546164C00F023FA002824D160781A
:101B70004101201D465C1E2E00DD1E262E706D1CB0
:101B8000701CC6B2002709E060784101201D0918C9
:101B9000781C085C28706D1C781CC7B2B742F3DB58
:101BA0006078401C60706078142801DB0020607051
:101BB00000210298017002E0022102980170FEBD2E
:101BC000C402002070B50025464C40214648FFF76E
:101BD000C1FE002839D00520C00120180079002856
:101BE00027DD0520C00120180079401E0521C9010C
:101BF000611808710520C00120188079FA2804DBDB
:101C000000200521C901611888710520C001201834
:101C100082790520C00120188079401C0523DB0152
:101C2000E318987131482018815C2F48FFF73FFF77
:101C300007E00520C001201840790521C90161187D
:101C4000887140212848FFF777FE20212648FFF7BA
:101C500081FE002844D02448FFF724FFC5B2244861
:101C60000078002802D0012831D107E0242D02D1CC
:101C700001201F4908700120E0702CE0232D17D1AE
:101C8000232120784201201D1018E2788154E17848
:101C900020784201201D81542078401C207020783B
:101CA000142801DB002020700020114908700DE08D
:101CB000242D02D10120E07008E020784101201D90
:101CC0000818E1784554E078401CE07003E00020FB
:101CD0000749087000BF00BF20210348FFF72CFE12
:101CE00070BD0000C40200200038014087020000DF
:101CF00041000020F8B505460E46344C002E01D1B7
:101D00000420F8BD00F054F9074625E00520C00185
:101D100020180079401C0521C901611808710520AF
:101D2000C00120184079FA2804DB00200521C901F0
:101D30006118487128780521C9016118497905227F
:101D4000D201A2185279521C0523DB01E3185A7103
:101D50001F4AA21850546D1C3046711ECEB2002886
:101D6000D4D1002F30D00520C001201800790028E0
:101D700008D00520C00120180079401E0521C901A6
:101D8000611808710520C00120188079FA2804DB49
:101D900000200521C901611888710520C0012018A3
:101DA00080790522D201A2189279521C0523DB0109
:101DB000E3189A71064AA218115C0648FFF777FEED
:101DC00008210448FFF7B8FD00209AE7C40200206C
:101DD000870200000038014030B47446641E257844
:101DE000641CAB4204D3635D5B00E31830BC18474E
:101DF0001D46F8E700F0BEF800F096F800F08EF807
:101E000000F07CF800F068F82EE0FEF7A7FE174817
:101E100000780F2805DB002014490870FEF71CFB32
:101E200022E013480078232807DB002010490870BF
:101E3000FEF7DAFAFEF7ACFE16E00E4800786428EA
:101E400009DB00200B490870FFF708FAFEF7E4FCF5
:101E5000FEF7AAFF08E008480078232803DB0020EB
:101E60000549087000E000BFCFE700003200002005
:101E700033000020340000203500002000210448F9
:101E80000178405C232801D1012070470020FCE745
:101E90004806002070B5054600240026E9000C4ADB
:101EA0005058FEF77BF9C6B200BF0CE0E8000849C5
:101EB0000858015D601C074A105C814201D0002077
:101EC00070BD601CC4B2B442F0DB0120F8E7000032
:101ED000F42400084806002010B50748FEF752FE1B
:101EE0000520FEF743FE7D20C000FEF745FEFEF70D
:101EF00035FEFEF72BFE10BD5555000000B58BB02A
:101F000001A8FFF79BFA0121684641701B2101706F
:101F100001218170FFF726F80BB000BD10B5FEF768
:101F2000F5FCFFF7C9FD10BD10B57D21C9000E48B5
:101F30000068FEF775F90446601E0C49884201D915
:101F400001200CE0601E0A4948610321081FFFF7C9
:101F50007DF80020064988610720086100200028DC
:101F600001D000BFFEE710BD00000020FFFFFF0012
:101F700000E000E010B50020094908700949087028
:101F80000949087009490870FFF71EFAFEF7E4FED8
:101F9000FEF77EFAFEF741FCFFF7E2F810BD000005
:101FA00032000020330000203400002035000020E3
:101FB0000448007803494978884201D101207047DC
:101FC0000020FCE7C402002003480021017041709A
:101FD0008170C17070470000C402002010B50A482B
:101FE0004079492805D1002202211046FFF7C4F8A4
:101FF00008E005484079562804D100220321104604
:10200000FFF7BAF810BD0000480600200B488079A1
:10201000302803D100210A48C1710EE007488079B9
:10202000312803D101210648C17106E003488079B7
:10203000322802D102210248C171704748060020AF
:10204000D00600200A48407A3038C1B2094881756C
:102050000748807A3038C1B20648163041700448CB
:10206000C07A3038C1B20348163081707047000022
:1020700048060020B0060020704710B5002202215B
:102080001046FFF779F810BD704700000248807ACB
:10209000302800D000BF70474806002010B58D489A
:1020A000407930380300FFF797FE05043A70A6DC4C
:1020B00039008849C97930390A225143854A127A50
:1020C000303A891808026421FEF7B4F8C1B2824898
:1020D000C1728049497A30390A2251437D4A927A45
:1020E000303A891808026421FEF7A4F8C1B27A4890
:1020F00001737849C97A30390A225143754A127BF3
:10210000303A891808026421FEF794F8C1B2724887
:102110008172007C012108436F490874D7E06D4942
:10212000C97930390A2251436A4A127A303A8918F9
:1021300008026421FEF77EF8C1B2674881736549E1
:10214000497A30390A225143624A927A303A8918E0
:1021500008026421FEF76EF8C1B25F48C1735D49A1
:10216000C97A30390A2251435A4A127B303A8918C7
:1021700008026421FEF75EF8C1B257484173007C43
:102180000221084354490874A1E05249C979303901
:102190000A2251434F4A127A303A891808026421C0
:1021A000FEF748F8C1B24C4881704A49497A303943
:1021B0000A225143474A927A303A89180802642128
:1021C000FEF738F8C1B24448C1704249C97A303983
:1021D0000A2251433F4A127B303A8918080264218F
:1021E000FEF728F8C1B23C484170007C0421084346
:1021F000394908746BE03749C97930390A225143AB
:10220000344A127A303A891808026421FEF712F82B
:10221000C1B2314841712F49497A30390A225143BC
:102220002C4A927A303A891808026421FEF702F8A3
:10223000C1B2294881712749C97A30390A225143EC
:10224000244A127B303A891808026421FDF7F2FF14
:10225000C1B221480171007C082108431E4908745D
:1022600035E01C49C97930390A225143194A127A9A
:10227000303A891808026421FDF7DCFFC1B2164824
:1022800001721449497A30390A225143114A927A2B
:10229000303A891808026421FDF7CCFFC1B20E481C
:1022A00041720C49C97A30390A225143094A127BDA
:1022B000303A891808026421FDF7BCFFC1B2064814
:1022C000C171007C102108430349087400BF00BF9E
:1022D00010BD000048060020B006002000200C4978
:1022E00089793039C8B2002804D109490A7A0949E4
:1022F000CA740CE0012805D105490A7A0549133151
:102300004A7004E002490A7A024913318A70704720
:1023100048060020B00600200B484079302803D141
:1023200000210A4841740EE007484079312803D162
:1023300001210648417406E003484079322802D161
:10234000022102484174704748060020B006002070
:10235000002002490870024948707047B40200200A
:10236000900600200020024908700249487070471A
:10237000B4020020900600200020054989793039F8
:10238000C8B2022800DD02200249887470470000AC
:1023900048060020B006002070B50646002400253F
:1023A0000E4C24202070641C49202070641C4420A2
:1023B0002070641C2C202070641C00BF01E0681C8D
:1023C000C5B20F2DFBDB31202070641C2320207050
:1023D000641C15210148FFF78DFC70BD66060020C6
:1023E00070B505460024264C24202070641C4B2028
:1023F0002070641C45202070641C59202070641CCF
:102400002812082803D13B202070641C18E02812F1
:10241000092803D13C202070641C11E028120A28EE
:1024200003D13D202070641C0AE028120B2803D140
:102430003E202070641C03E0281230302070641CA1
:102440002C202070641C01210E48017228120528DE
:1024500007DAE8B2022804D1FF200002054001207B
:102460000543284630302070641C2846FEF776FC71
:1024700023202070641C09210148FFF73BFC70BD3C
:1024800066060020D006002000BF704770B50646E3
:10249000002400250F4C24202070641C562020703E
:1024A000641C2C202070641C00BF05E00A48405DBD
:1024B0002070641C681CC5B20F2DF7DB462020700D
:1024C000641C23202070641C14210248FFF712FCB6
:1024D00070BD000066060020DC240008535A443119
:1024E00030313031323231303233300024484541DE
:1024F00052540000C025000879200008A8250008D3
:10250000512300088C250008652300086C2500086D
:1025100089200008702500089D20000880250008FB
:1025200079230008C8250008DD220008A42500083A
:1025300019230008882500087B200008782500085A
:10254000452000089C2500080D200008982500085B
:10255000DD1F0008B42500088D200008892400082C
:10256000E1230008992300088D2400084D49430009
:102570004E4C454400000000444F4F524C4544002F
:10258000554C454400000000494400005359535540
:10259000504441544500000041534B0043414C4CD2
:1025A00000000000534950005359535245534554BD
:1025B000000000004E4554524553455400000000B1
:1025C000484541525400000052454C41590000001A
:1025D0000830000800000020680000000401000826
:1025E0007030000868000020D80C000020010008AE
:1025F00000000000000000000000000000000000DB
:1026000000000000000000000000000000000000CA
:1026100000000000000000000000000000000000BA
:1026200000000000000000000000000000000000AA
:103000004632303800000000006CDC020000000096
:103010000000000001020304060708090000000088
:1030200000000000000000000000000000000000A0
:103030000000000000000000000000000000000090
:10304000000000000000000000000000C0A801D344
:10305000C0A801010000C0A801AA000000000000F3
:10306000000000000102030401020304060708092E
:04000005080000C12E
:00000001FF
